:020000040000FA
:100000000C2882073F3406345B344F3466346D3439
:100010007D3407347F346F3483160C3085008601BD
:100020008312803081008601A401A501A60107305A
:100030009F0044280A30A1000000A00B1C28A10B3F
:100040001C280034261900342615A40A0A30240678
:10005000031D0034A401A50A0A3025060319A501D1
:100060000034A6190034A615A403FF302406031D8E
:1000700000340930A400A503FF30250603194128E8
:100080000034A501A4010034051D2220851D312066
:10009000013085002408012086001A2086010230E4
:1000A00085002508012086001A20860105192611E1
:0600B0008519A611442889
:02400E00503F21
:00000001FF
